:100000000C94D6030C94F3030C94F3030C94F303B5
:100010000C94F3030C94F3030C94F3030C94F30388
:100020000C94F3030C94F3030C945A0A0C94F3030A
:100030000C94F3030C94A01C0C94F3030C94CD1CAF
:100040000C94F3030C94F3030C94F3030C94F30358
:100050000C94F30354797065202268656C7022203B
:10006000666F7220636F6D6D616E64206C6973746E
:100070002E0031303A35333A303600417567203240
:100080003620323030390048656174696E6700553A
:100090006E6B6E6F776E004F6666004175746F6DA4
:1000A00061746963004D616E75656C6C204F6E0004
:1000B0004C6561726E004C6561726E205265666CB3
:1000C0006F772054656D700000234D6F6465203A92
:1000D00020002C20002C20002C2000235365746964
:1000E0006E672054656D70206F66667365740023BB
:1000F0004572726F722054656D7020646966662067
:10010000746F6F2068696768002064656743290021
:1001100020280020202054203D20200029202020BD
:10012000546F6C64203D20200020280020202054A3
:10013000203D2020004454203D20004F76657273FE
:10014000686F6F74203D2000005806880400001C72
:10015000050B14060BA704050C0506FC040AEC04A9
:10016000010000000000000000000000000155092F
:10017000CA0751081C050BF40400D3040200000157
:10018000000000000000000000000000000000006F
:100190000000021C09C70749081C050BF40400D322
:1001A0000403000002000000000000000000000046
:1001B0000000000000000003DE08C40741081C0521
:1001C0000BF40400D30404980404000003000000AE
:1001D00000000000000000000000000004A508C1AD
:1001E0000739081C050BF40400D3040500000400C3
:1001F00000000000000000000000000000000000FF
:1002000000052608BE0789041C050BC80400000071
:1002100005000000000000000000000000000000D9
:10022000000000000000064606BB078D041C050BFD
:10023000140500B2040700000600000000000000E2
:100240000000000000000000000000071308B807CD
:100250000F081C050B140500A70408000007000088
:10026000000000000000000000000000000000008E
:1002700008E407B5072B061C050B140500BD04098F
:100280000000080000000000000000000000000066
:10029000000000000009EC05B20759081C050B140A
:1002A00005008F04000000090000000000000000AD
:1002B000000000000000000000000ACD07AF076C3E
:1002C000061C050B04050000000A000000000000E9
:1002D0000000000000000000000000000000000B13
:1002E0001C06FC058E041C050B0C0506FC040A14F8
:1002F000060B0000000000000000000000000000ED
:1003000000000000205472616E73203A200020002B
:10031000205374617465203A200068656C70006831
:10032000696C66650073686F77616C6C001A0337DF
:1003300006F0181F033706F0182503320786142A23
:10034000050000A717320500006B173A0500002EC4
:100350001741050000F1164A050000B516530500C7
:100360000078165B0500003B1666050000FF15715E
:10037000050000C2157B05000085158505000049B4
:10038000158F0500000C151F050000D314980550AB
:1003900006EC18A1059A06E8180A050000321810A4
:1003A0000500000818F6040000FC17FA04AB05F479
:1003B00017FF04C005EC170505D205E41716050064
:1003C000005C18000000000000232020436F6D6DCA
:1003D000616E6473203A20002320757365202268C3
:1003E000656C7022002320436F6D6D616E64206E1A
:1003F0006F7420666F756E64003031323334353679
:1004000037383941424344454600504342502D520B
:1004100065666C6F7720436F6E74726F6C6C65727B
:1004200000536F66747761726520004461746520C3
:100430003A200054696D65203A200073746172742B
:1004400020007265616479200073656C6674657361
:100450007420002064656743002053656B756E64EB
:10046000656E002025002050686173656E6D6F64B5
:10047000757300204F4E00204F464600204C6561AA
:10048000726E0020507265686561740020536F6160
:100490006B00204477656C6C00205265666C6F774A
:1004A000002054656D706572617475723A00205A4F
:1004B0006569743A0020416E73746965673A00207B
:1004C0004C65697374756E673A00205B30206F6409
:1004D000657220315D00205B302E2E3235345D0098
:1004E000205B302E2E36353533345D00205B302EC8
:1004F0002E3130305D0070656300736F6C64006C8A
:100500006561726E0073746F700064656275670078
:1005100074726163650073657474696E67730074E7
:10052000656D706F66667365740070687474656D70
:10053000700070687474696D6500706874707772AB
:1005400000736F616B74656D7000736F616B7469BC
:100550006D6500736F616B707772007265666C6FAA
:100560007774656D70007265666C6F7774696D6520
:10057000007265666C6F77707772006477656C6C7B
:1005800074656D70006477656C6C74696D6500648A
:1005900077656C6C7077720074656D7073686F77D7
:1005A0000074656D707472616365002053746172CC
:1005B000746574204C6F6574766F7267616E670046
:1005C0002053746172746574204C65726E6C617531
:1005D00066002053746F7074204C6F6574766F7270
:1005E00067616E67002053656C656B746965727432
:1005F0002064656E20616B746976656E205061724F
:10060000616D657465727361747A205B20302E2E83
:1006100034205D002054656D7065726174757220C0
:100620004A757374616765205B2D33302E2E33302D
:100630005D204772616400204C69737465742061A9
:100640006C6C652042656665686C65206175660046
:100650002054656D7065726174757220696E206AD0
:100660006564657220506861736520616C6C6572A9
:1006700020582053656B756E64656E2061757367D5
:100680006562656E205B506172616D657465722094
:1006900030206F64657220585D002054656D706570
:1006A00072617475722077C3A46872656E64206489
:1006B0006573204CC3B674656E7320616C6C657293
:1006C00020582053656B756E64656E206175736785
:1006D0006562656E205B506172616D657465722044
:1006E00030206F64657220585D0020446562756734
:1006F00067696E6720496E666F726D6174696F6EAF
:10070000656E2020617573676562656E0020496EB5
:100710007465726E65204175746F6D6174656E7A73
:1007200075737461656E6465206175736765626574
:100730006E0020416C6C652045696E7374656C6C4D
:10074000756E67656E20617573676562656E002002
:100750002D2D3E20000D0A4175746F6D6174697313
:1007600063686572204C6F65746265747269656256
:10077000206E6F6368206E69636874206D6F6567B3
:100780006C6963682E0D0A42697474652065727322
:1007900074204F66656E706172616D65746572205C
:1007A00065696E6C65726E656E0D0A0011241FBE60
:1007B000CFE5D8E0DEBFCDBF10E0A0E6B0E0E2E0DC
:1007C000F5E402C005900D92A03BB107D9F712E005
:1007D000A0EBB0E001C01D92A437B107E1F70E9481
:1007E000F5030C947F220C9400000E94C2090E9421
:1007F0002C1E0E94F50B0E94EA0A0E94FF1960E875
:1008000075E280E090E00E94491D8EE19DE10E942A
:100810007914789460E875E280E090E00E945E1CB4
:100820008DE79CE10E94561B8AE094E00E94931B96
:1008300081E294E00E94731B8BE294E00E94731BA0
:100840008BE790E00E94731B0E94861B81E294E07C
:100850000E94731B83E394E00E94731B82E790E085
:100860000E94731B0E94861B0E9465120E949C09B5
:1008700081E00E94431B80E00E94171B89E494E002
:100880000E94731B8BE394E00E94931B0E940D1E39
:1008900082E00E94961D88EE93E00E943A1A882317
:1008A000D1F70E94961D89E494E00E94731B82E4B4
:1008B00094E00E94931B84E590E00E94731B0E94C9
:1008C000861B0E943B050E94330B80E00E94C10BF7
:1008D000882359F00E942405833011F484E003C07A
:1008E0000E94A20A82E00E941F0581E00E94C10BC3
:1008F000882319F081E00E941F0582E00E94C10B4D
:10090000882319F083E00E941F050E94EA19D9CFBD
:10091000089581E08093B60008950895089520E039
:1009200080910A0290910B0297FD21E0822F089599
:1009300040E02091CF003091D0008091D100909183
:10094000D200281739070CF041E0842F089520E0E9
:100950008091CF009091D000883C91050CF021E06F
:10096000822F089520E08091CF009091D000893CA3
:1009700091050CF421E0822F089520E08091CF00B2
:100980009091D000805991400CF021E0822F089581
:1009900020E08091CF009091D000883C91050CF42C
:1009A00021E0822F089560E02091BB003091BC00CF
:1009B0004091BD005091BE008091BF009091C00059
:1009C000A091C100B091C200281739074A075B0700
:1009D00008F061E0862F089590E08091B5008230A4
:1009E00009F491E0892F089590E08091B50082305C
:1009F00009F091E0892F089590E08091B50084304E
:100A000009F491E0892F089590E08091B500843039
:100A100009F091E0892F089590E08091B50083302E
:100A200009F491E0892F089590E08091B50083301A
:100A300009F091E0892F08958091B00008958530E4
:100A400010F48093B60008958091B50008951F9327
:100A5000182F0E94660F882329F08091D300612F00
:100A60000E944C0E1F9108950E94101A9093D0007E
:100A70008093CF000895EF92FF920F931F930E94EF
:100A8000DF0A7B018C018091BB009091BC00A0919A
:100A9000BD00B091BE008E159F05A007B10709F4F7
:100AA0005AC0E092BB00F092BC000093BD001093CE
:100AB000BE0080E090E00E943A1A8093B0000E944D
:100AC000E30F882309F447C08091B100882319F00F
:100AD00081508093B1008091B1008823E1F50E949C
:100AE000FC0F882339F08091600090916100875756
:100AF000944089F180916000909161000E94731B85
:100B000088ED90E00E94731B0E94E30F8093B10078
:100B10008AE066E040E020E20E94981B85ED90E0CC
:100B20000E94731B0E94101A64E070E00E94F8217A
:100B30007B010027F7FC0095102F8AE064E041E07C
:100B400020E30E94981B82ED90E00E94731B83E5D6
:100B500094E00E94931B8091B7009091B80090930D
:100B6000BA008093B90062E670E043ED50E00E9465
:100B7000850C9093B8008093B7002091B900309114
:100B8000BA002817390719F080E00E9427059091D4
:100B9000B6008091B5008917D1F09093B5000E94FE
:100BA0007F0F8823A1F089EC90E00E94731B809155
:100BB000B50090E0FC01EE0FFF1FE80FF91FEA56A9
:100BC000FF4F818192810E94731B0E94861B1F919F
:100BD0000F91FF90EF9008958CE794E0909361005F
:100BE0008093600089E00E94961D88E290E09093D7
:100BF000CE008093CD0008958091B000882341F00D
:100C00000E94931D823079F082E00E94961D089523
:100C10000E94CA0F8F3F39F40E94931D813019F052
:100C200081E00E94961D08950E94CA0F90E08F3FB8
:100C300009F491E0892F089587E794E0909361008B
:100C4000809360000E94111B80E00E94961D81E04D
:100C50008093B60008958091BB009091BC00A09154
:100C6000BD00B091BE008093C7009093C800A093D0
:100C7000C900B093CA0080910A0290910B02909330
:100C80000902809308020E94111B08958CE794E0EA
:100C900090936100809360000E94111B89E00E9484
:100CA000961D88E290E09093CE008093CD00089549
:100CB00087E794E090936100809360000E94111B8D
:100CC00080E00E94961D0E94CA0F80930C028F3F05
:100CD00011F410920C020895EF92FF920F931F935C
:100CE0000E94111B0E947F0F882379F183E191E01C
:100CF0000E94731BE090CF00F090D0000027F7FC1B
:100D00000095102F8AE064E041E020E20E94981BE9
:100D100080E191E00E94731B8091CF009091D00000
:100D200064E070E00E94F8217B010027F7FC009549
:100D3000102F8AE064E041E020E20E94981B89E0E5
:100D400091E00E94731B0E94861B81E08093B50096
:100D50008093B6000E948B11282F30E0220F331FA2
:100D6000220F331F8091CF009091D000281B390BA8
:100D7000C90182589F4F79010027F7FC0095102F79
:100D80008D3F910538F088EB9BE00E94061E8FEEA8
:100D900090E005C0822F0E94BA0F8BED90E00E9478
:100DA000731B8AE064E041E020E20E94981B0E94ED
:100DB000861B1F910F91FF90EF900895EF92FF9285
:100DC0000F931F938091B2009091B300892B41F44F
:100DD0008091CF009091D0009093B3008093B200A7
:100DE0000E94C90A9091B400882309F489C099230C
:100DF00009F48BC08091CF009091D0002091B20077
:100E00003091B300821B930B29E130E0AC01429F8B
:100E1000C001439F900D529F900D112440910A02F2
:100E200050910B029A01220F331F240F351F820F9E
:100E3000931F64E070E00E94F82170930B026093AE
:100E40000A021092B4000E947F0F882309F44FC059
:100E500085E391E00E94731BE0900A02F0900B0280
:100E60000027F7FC0095102F8AE064E041E020E2C3
:100E70000E94981B8CE291E00E94731BE090CF00CF
:100E8000F090D0000027F7FC0095102F8AE064E076
:100E900041E020E20E94981B89E291E00E94731BCE
:100EA0008091CF009091D00064E070E00E94F82122
:100EB0007B010027F7FC0095102F8AE064E041E0F9
:100EC00020E20E94981B8CE191E00E94731BE0904D
:100ED000B200F090B3000027F7FC0095102F8AE0D5
:100EE00064E041E020E20E94981B0E94861B8091F2
:100EF000CF009091D0009093B3008093B20005C0D2
:100F0000992319F481E08093B40080910C0290E061
:100F100020910A0230910B02AC01429FC001439F15
:100F2000900D529F900D112464E670E00E94F8210C
:100F30008091CF009091D000860F971F2091CD0017
:100F40003091CE00821793071CF40E940C1B02C044
:100F50000E94111B1F910F91FF90EF9008950E9426
:100F6000DE0608950E94DE0608950E94DE060895BA
:100F70000E94DE0608950E94DE0608950E94DE06A5
:100F800008950E94DE0608950E94DE0608950E94DC
:100F9000DE0608950E94DE0608958CE794E09093A3
:100FA00061008093600084E60E94171B80EB94E050
:100FB0009093CE008093CD0084E00E94961D88EE31
:100FC00093E00E94061E08958CE794E090936100E0
:100FD0008093600089E00E94961D10920B0210928F
:100FE0000A0210920902109208028091BB009091AF
:100FF000BC00A091BD00B091BE008093C30090934F
:10100000C400A093C500B093C60088E092E090931E
:10101000CE008093CD0084E60E94171B089580E0E7
:101020000E94171B08958CE794E0909361008093D1
:10103000600089E00E94961D88E092E09093CE00C7
:101040008093CD0084E60E94171B089587E794E003
:10105000909361008093600080E00E94171B88ECF1
:1010600090E09093CE008093CD0083E00E94961D87
:10107000089580E00E94171B80EA9FE00E94061EF0
:10108000089580E00E94171B84E690E00E94061EEF
:10109000089580E00E94171B84E690E00E94061EDF
:1010A000089580E00E94171B84E690E00E94061ECF
:1010B0000895EF92FF920F931F936091CF0070916C
:1010C000D000882777FD8095982F29E130E040E017
:1010D00050E00E94C52160517742804090402091AD
:1010E000080230910902442737FD4095542F0E9491
:1010F0002D2220930C020E947F0F882389F08BE31E
:1011000091E00E94731BE0900C02FF2400E010E0CD
:101110008AE064E041E020E20E94981B0E94861B66
:1011200080E00E94171B88EE93E00E94061E8091CB
:101130000C020E94D30F81E08093B5008093B6002B
:101140001F910F91FF90EF900895EF92FF920F93F0
:101150001F9382E994E090936100809360000E9465
:101160003A110E94171BE090BB00F090BC00009168
:10117000BD001091BE000E940712A0E0B0E08E0DED
:101180009F1DA01FB11F8093BF009093C000A0932C
:10119000C100B093C2000E941C1190E0880F991FFB
:1011A000880F991F9093CE008093CD0088E00E9415
:1011B000961D1F910F91FF90EF900895EF92FF926F
:1011C0000F931F930E94A9110E94171BE090BB0070
:1011D000F090BC000091BD001091BE000E94FA1179
:1011E000A0E0B0E08E0D9F1DA01FB11F8093BF0037
:1011F0009093C000A093C100B093C2000E948B11D5
:1012000090E0880F991F880F991F9093CE008093CC
:10121000CD000E948B1190E0880F991F880F991FB5
:101220009093D2008093D10087E00E94961D1F9179
:101230000F91FF90EF900895EF92FF920F931F93FD
:101240008CE894E090936100809360000E94CB1042
:101250000E94171BE090BB00F090BC000091BD0005
:101260001091BE000E941412A0E0B0E08E0D9F1DF0
:10127000A01FB11F8093BF009093C000A093C10036
:10128000B093C2000E94AD1090E0880F991F880FA4
:10129000991F9093CE008093CD0086E00E94961D0A
:1012A0001F910F91FF90EF900895EF92FF920F938F
:1012B0001F9383E894E090936100809360000E9404
:1012C000A20A1092BB001092BC001092BD001092B6
:1012D000BE000E9452100E94171BE090BB00F090CD
:1012E000BC000091BD001091BE000E942112A0E040
:1012F000B0E08E0D9F1DA01FB11F8093BF00909383
:10130000C000A093C100B093C2000E94321090E0D0
:10131000880F991F880F991F9093CE008093CD005E
:1013200085E00E94961D84E690E00E94061E1F91B3
:101330000F91FF90EF90089581E08093B500809326
:10134000B60082E690E063ED70E047E850E00E946E
:10135000510D9093B8008093B70080E00E9427055C
:101360000E94600FBC0184E395E00E940F0A9093F5
:10137000CC008093CB000E94101A9093D0008093F1
:10138000CF000895E4EDF0E011821082379681E0FD
:10139000EA31F807C9F787E48CBF83B78D6083BF54
:1013A00089B7826089BF0895CF93DF93EC01A4EDE4
:1013B000B0E0E0E0F0E08D919C911197892B21F550
:1013C0009F0193E0EE0FFF1F9A95E1F7E21BF30BED
:1013D000EC52FF4F168213821282CB0105966AE00F
:1013E00070E00E94E42175836483F894F90183E03E
:1013F000EE0FFF1F8A95E1F7E21BF30BEC52FF4F54
:10140000D183C083789407C031961796EA30F105EE
:1014100091F62FEF3FEFC901DF91CF910895CF9360
:10142000DF93EC01A4EDB0E0E0E0F0E08D919C9161
:101430001197892B29F59F0153E0EE0FFF1F5A9555
:10144000E1F7E21BF30BEC52FF4F81E0868313823E
:101450001282CB0105966AE070E00E94E421758358
:101460006483F894F90143E0EE0FFF1F4A95E1F71A
:10147000E21BF30BEC52FF4FD183C083789407C07B
:1014800031961796EA30F10589F62FEF3FEFC90143
:10149000DF91CF910895F894FC0163E0EE0FFF1FF8
:1014A0006A95E1F7E81BF90BEC52FF4F11821082AD
:1014B000789408951F920F920FB60F9211242F93D4
:1014C0003F934F935F936F937F938F939F93AF93CC
:1014D000BF93CF93DF93EF93FF93C4EDD0E0888168
:1014E0009981892BB9F08A819B8101969B838A839C
:1014F0002A813B818C819D812817390758F0E8812A
:10150000F98109958E81882319F01B821A8202C005
:1015100019821882279681E0CA31D80701F7FF9116
:10152000EF91DF91CF91BF91AF919F918F917F917B
:101530006F915F914F913F912F910F900FBE0F9040
:101540001F90189510921E0110921F0110922001F9
:1015500010922101089590E080911A01882309F4E6
:1015600091E090931A01992399F080911E01909136
:101570001F01A0912001B09121010196A11DB11D73
:1015800080931E0190931F01A0932001B09321012D
:10159000089580911A010895882371F080911B01AC
:1015A000882351F410921A0181E080931B01F89472
:1015B0001DBC1CBC7894089510921B010895F894EA
:1015C000789460911E0170911F018091200190918B
:1015D0002101089510921E0110921F011092200106
:1015E000109221018BEA9AE064EF71E00E940F0AE9
:1015F00090931D0180931C0110921A0181E0809349
:101600001B01F8941DBC1CBC7894089581E0809364
:101610002A010895E82FF0E0EE0FFF1FEE5DFE4F68
:101620008081662319F0880F816001C0880F808354
:10163000808190E08F709070009711F00F9791F477
:101640008181662341F080FD02C0856081838181B4
:101650008D7F8183089580FF02C0826081838181B4
:101660008A7F81830895EF92FF920F931F93809159
:101670002A01882339F110922A0100B3602F609566
:10168000661F6627661F80E00E940A0B10E0B80103
:1016900036E0769567953A95E1F721E0E22EF12C58
:1016A0006E257F25617081E00E940A0B95E01695FA
:1016B00007959A95E1F70E251F25017082E0602FAE
:1016C0000E940A0B1F910F91FF90EF900895E82F51
:1016D000F0E0EE0FFF1FEE5DFE4F818181700895F7
:1016E000809128019091290101969093290180937E
:1016F0002801039720F010922901109228012091CF
:1017000028013091290140E050E02F5F3F4F233006
:10171000310510F020E030E0922FE22FF0E0EE0FE4
:10172000FF1FEE5DFE4F818180FF06C030932901CF
:1017300020932801892F08954F5F5F4F4330510553
:1017400021F7309329012093280194E0F3CFE82F6B
:10175000F0E0EE0FFF1FEE5DFE4F818190E0969569
:1017600087959695879581700895E82FF0E0EE0FA4
:10177000FF1FEE5DFE4F818190E096958795817009
:101780000895E82FF0E0EE0FFF1FEE5DFE4F218180
:10179000822F90E09695879596958795982F9170D2
:1017A00080FF02C02B7F2183892F0895E82FF0E06E
:1017B000EE0FFF1FEE5DFE4F2181822F90E0969588
:1017C0008795982F917080FF02C02D7F2183892FEC
:1017D0000895E82FF0E0EE0FFF1FEE5DFE4F8181D0
:1017E000856081838FE08083089581B38F7181BB91
:1017F00082B3806E82BB109222011092230110925C
:1018000024011092250110922601109227011092B6
:1018100029011092280110922A0186E09BE06AE0DB
:1018200070E00E940F0A90932C0180932B01089581
:10183000DF93CF93CDB7DEB72E970FB6F894DEBF08
:101840000FBECDBF20E030E0AE014F5F5F4FFC0127
:10185000E20FF31FE491DA01A20FB31FEC932F5FA5
:101860003F4F2730310599F7DE011896FA0187E0DE
:1018700001900D928150E1F7288539854A855B8575
:101880006C857D858E8590E02E960FB6F894DEBF30
:101890000FBECDBFCF91DF910895DF93CF9300D0DE
:1018A00000D000D0CDB7DEB7FC018491898331969A
:1018B00084918A833196E491EB83DE011496FE01D4
:1018C000319683E001900D928150E1F76C817D812A
:1018D0008E8190E026960FB6F894DEBF0FBECDBF86
:1018E000CF91DF91089580E0089580E0089580E031
:1018F000089582E00E94C10B089581E00E94C10B0F
:10190000089580E00E94C10B08953F924F925F922C
:101910006F927F928F929F92AF92BF92CF92DF92FF
:10192000EF92FF920F931F93DF93CF93CDB7DEB764
:10193000A2970FB6F894DEBF0FBECDBF5C012B019E
:101940003A01FC01028113812081318180E090E025
:10195000AE01495F5F4FF901E80FF91FE491DA0129
:10196000A80FB91FEC93019687309105A1F7DE010E
:101970001E96FA0187E001900D928150E1F72989C6
:101980003A893E848B889C88F801849189830F5F13
:101990001F4FF80184918A830F5F1F4FF8018491D4
:1019A000025010408B83E980FA80D82E2115310532
:1019B00011F0F9010995CC24C394E114F10429F044
:1019C000F7010995882309F43CC0D31409F44FC0EA
:1019D0008114910411F0F40109950D2D10E0000F10
:1019E000111F000F111F040D151DF80120813181F9
:1019F00080E090E0AE014B5E5F4FF901E80FF91F08
:101A0000E491DA01A80FB91FEC9301968730910594
:101A1000A1F7DE015C96FA0187E001900D928150FA
:101A2000E1F7FC8CED8DFE8D309709F0099561147E
:101A30007104F1F0F30180816F2D4C2D0E942A0E6C
:101A400017C00D5F1F4FF80184918C830F5F1F4FEC
:101A5000F80184918D830F5F1F4FF801849102502C
:101A600010408E83C394EC80FD80D82EA6CF8501D4
:101A7000C801A2960FB6F894DEBF0FBECDBFCF91BE
:101A8000DF911F910F91FF90EF90DF90CF90BF906B
:101A9000AF909F908F907F906F905F904F903F900E
:101AA0000895AF92BF92CF92DF92FF920F931F9350
:101AB000DF93CF93CDB7DEB765970FB6F894DEBF4F
:101AC0000FBECDBF8C016B015A01FC012081318119
:101AD00080E090E0AE01485F5F4FF901E80FF91F29
:101AE000E491DA01A80FB91FEC93019687309105B4
:101AF000A1F7DE011F96FA0187E001900D92815057
:101B0000E1F7DE011196FE013F9687E001900D920C
:101B10008150E1F7EA81FB81F980309709F009955E
:101B2000C114D10431F08F2DB5010E94CE0DF60104
:101B30008083C80165960FB6F894DEBF0FBECDBF97
:101B4000CF91DF911F910F91FF90DF90CF90BF90C9
:101B5000AF90089510922E0110922D011092420123
:101B600010924101109256011092550110926A0193
:101B70001092690110927E0110927D010895EDE2AC
:101B8000F1E020E080819181892B09F02F5F74962C
:101B900081E0E139F807B1F7822F0895482F6115E8
:101BA000710509F43FC0EDE2F1E020E030E0808112
:101BB0009181892B89F584E190E0289FD001299FAC
:101BC000B00D389FB00D1124A35DBE4F11967C93CC
:101BD0006E93F901EE0FFF1FC90163E0880F991F93
:101BE0006A95E1F7E80FF91FEE0FFF1FE15DFE4F69
:101BF00081E08083FD011382F901EE0FFF1FEE0FDC
:101C0000FF1FE20FF31FEE0FFF1FEE0FFF1FEF5C32
:101C1000FE4F4083822F08952F5F3F4F74962530EB
:101C2000310529F68FEF08958F3F99F085308CF4B8
:101C3000282F332727FD309584E190E0289FF0017D
:101C4000299FF00D389FF00D1124E35DFE4F1182A6
:101C500010820895E82F8F3FF1F08530E4F484E19D
:101C6000E802D0011124A35DBE4FFD018381E80F7E
:101C7000F11D44878F5FFD018383883009F413824F
:101C8000FD018281883010F48F5F8283FD018381A2
:101C9000E80FF11D64830895AF92BF92CF92DF9257
:101CA000EF92FF920F931F93DF93CF93CDB7DEB7E1
:101CB0006E970FB6F894DEBF0FBECDBF482F8F3F93
:101CC00009F4CBC085300CF0C8C0282F332727FD7E
:101CD000309584E190E0289FF001299FF00D389F16
:101CE000F00D1124E35DFE4F80819181892B09F471
:101CF000B4C084E1480280011124035D1E4FF80145
:101D0000808191810E94731B80E193E00E94731B8C
:101D1000F8018281883010F4FF2403C0F801F380B9
:101D2000F3941982EE246E010894C11CD11CF8EAC8
:101D3000AF2EF0E0BF2E2CC0F8E0FF1609F4FF2410
:101D4000F801EF0DF11D8481F3942DB73EB72850B3
:101D500030400FB6F8943EBF0FBE2DBFADB7BEB733
:101D60001196EDB7FEB7D282C182FD01B382A28285
:101D7000D582C482868317820E94241FE3942DB7E4
:101D80003EB7285F3F4F0FB6F8943EBF0FBE2DBF42
:101D9000F8018281E81680F2CE0101960E94611B53
:101DA0008EE093E00E94731BF8018281882309F47E
:101DB00052C0883010F4FF2403C0F801F380F3947C
:101DC0001982EE24E3946E010894C11CD11CE8EA48
:101DD000AE2EE0E0BE2E2CC0F8E0FF1609F4FF2482
:101DE000F801EF0DF11D8485F3942DB73EB728500F
:101DF00030400FB6F8943EBF0FBE2DBFADB7BEB793
:101E00001196EDB7FEB7D282C182FD01B382A282E4
:101E1000D582C482868317820E94241FE3942DB743
:101E20003EB7285F3F4F0FB6F8943EBF0FBE2DBFA1
:101E3000F8018281E81680F20E94861BF8018081F9
:101E400091810E94731B84E093E00E94731BCE017A
:101E500001960E94611B0E94861B6E960FB6F89435
:101E6000DEBF0FBECDBFCF91DF911F910F91FF90CD
:101E7000EF90DF90CF90BF90AF9008959C01E199D3
:101E8000FECF3FBB2EBBE09A8DB308959C01E19934
:101E9000FECF3FBB2EBB6DBB0FB6F894E29AE19A22
:101EA0000FBE08959C01E199FECFE199FECF3FBBA3
:101EB0002EBB6DBB0FB6F894E29AE19A0FBE08955F
:101EC00088EC90E0089582E090E00895E199FECFDB
:101ED00089E690E09FBB8EBBE09A8DB30895282FD2
:101EE000E199FECFE199FECF89E690E09FBB8EBBE2
:101EF0002DBB0FB6F894E29AE19A0FBE0895E199CE
:101F0000FECF8AE690E09FBB8EBBE09A8DB308952A
:101F1000282FE199FECFE199FECF8AE690E09FBBA2
:101F20008EBB2DBB0FB6F894E29AE19A0FBE0895CE
:101F3000E199FECF85E690E09FBB8EBBE09A8DB322
:101F40000895282FE199FECFE199FECF85E690E034
:101F50009FBB8EBB2DBB0FB6F894E29AE19A0FBEE1
:101F60000895E199FECF8DE690E09FBB8EBBE09A8D
:101F70008DB30895282FE199FECFE199FECF8DE62C
:101F800090E09FBB8EBB2DBB0FB6F894E29AE19A0E
:101F90000FBE0895E199FECF8EE690E09FBB8EBB09
:101FA000E09A8DB30895282FE199FECFE199FECFF5
:101FB0008EE690E09FBB8EBB2DBB0FB6F894E29AE5
:101FC000E19A0FBE0895E199FECF8BE690E09FBBAA
:101FD0008EBBE09A8DB30895282FE199FECFE19949
:101FE000FECF8BE690E09FBB8EBB2DBB0FB6F89467
:101FF000E29AE19A0FBE0895E199FECF8CE690E057
:102000009FBB8EBBE09A8DB30895282FE199FECF38
:10201000E199FECF8CE690E09FBB8EBB2DBB0FB647
:10202000F894E29AE19A0FBE0895E199FECF84E612
:1020300090E09FBB8EBBE09A8DB30895282F85302A
:1020400080F480939101E199FECFE199FECF84E67F
:1020500090E09FBB8EBB2DBB0FB6F894E29AE19A3D
:102060000FBE089590919101E199FECF8AE0989F6B
:10207000C0011124880F991F8E5F9F4F9FBB8EBB9D
:10208000E09A8DB3089590919101E199FECF84E19A
:10209000989FC00111248D5F9F4F9FBB8EBBE09A1C
:1020A0008DB3089590919101E199FECF85E0989FBD
:1020B000C0011124880F991F880F991F8C5F9F4FB3
:1020C0009FBB8EBBE09A8DB30895282F909191010C
:1020D000E199FECFE199FECF8AE0989FC0011124DB
:1020E000880F991F8E5F9F4F9FBB8EBB2DBB0FB676
:1020F000F894E29AE19A0FBE0895282F90919101E9
:10210000E199FECFE199FECF84E1989FC0011124AF
:102110008D5F9F4F9FBB8EBB2DBB0FB6F894E29A8D
:10212000E19A0FBE0895282F90919101E199FECF79
:10213000E199FECF85E0989FC0011124880F991F77
:10214000880F991F8C5F9F4F9FBB8EBB2DBB0FB617
:10215000F894E29AE19A0FBE089590919101E19965
:10216000FECF84E1989FC0011124895F9F4F9FBBE0
:102170008EBBE09A8DB3089590919101E199FECFC5
:1021800084E1989FC0011124885F9F4F9FBB8EBB45
:10219000E09A8DB3089590919101E199FECF84E189
:1021A000989FC0011124875F9F4F9FBB8EBBE09A11
:1021B0008DB30895282F90919101E199FECFE19977
:1021C000FECF84E1989FC0011124895F9F4F9FBB80
:1021D0008EBB2DBB0FB6F894E29AE19A0FBE08951C
:1021E000282F90919101E199FECFE199FECF84E1F2
:1021F000989FC0011124885F9F4F9FBB8EBB2DBB52
:102200000FB6F894E29AE19A0FBE0895282F9091A4
:102210009101E199FECFE199FECF84E1989FC00141
:102220001124875F9F4F9FBB8EBB2DBB0FB6F894C9
:10223000E29AE19A0FBE089590919101E199FECF43
:1022400084E1989FC00111248F5E9F4F9FBB8EBB7E
:10225000E09A8DB3089590919101E199FECF84E1C8
:10226000989FC00111248E5E9F4F9FBB8EBBE09A4A
:102270008DB3089590919101E199FECF84E1989FEB
:10228000C00111248D5E9F4F9FBB8EBBE09A8DB322
:102290000895282F90919101E199FECFE199FECF09
:1022A00084E1989FC00111248F5E9F4F9FBB8EBB1E
:1022B0002DBB0FB6F894E29AE19A0FBE0895282F2D
:1022C00090919101E199FECFE199FECF84E1989F31
:1022D000C00111248E5E9F4F9FBB8EBB2DBB0FB6DE
:1022E000F894E29AE19A0FBE0895282F90919101F7
:1022F000E199FECFE199FECF84E1989FC0011124BE
:102300008D5E9F4F9FBB8EBB2DBB0FB6F894E29A9C
:10231000E19A0FBE089590919101E199FECF84E179
:10232000989FC0011124845F9F4F9FBB8EBBE09A92
:102330008DB3089590919101E199FECF84E1989F2A
:10234000C0011124835F9F4F9FBB8EBBE09A8DB36A
:10235000089590919101E199FECF84E1989FC00189
:102360001124825F9F4F9FBB8EBBE09A8DB308956F
:10237000282F90919101E199FECFE199FECF84E160
:10238000989FC0011124845F9F4F9FBB8EBB2DBBC4
:102390000FB6F894E29AE19A0FBE0895282F909113
:1023A0009101E199FECFE199FECF84E1989FC001B0
:1023B0001124835F9F4F9FBB8EBB2DBB0FB6F8943C
:1023C000E29AE19A0FBE0895282F90919101E19928
:1023D000FECFE199FECF84E1989FC0011124825F76
:1023E0009F4F9FBB8EBB2DBB0FB6F894E29AE19A2C
:1023F0000FBE08958091910124E1829FC0011124B4
:10240000865F9F4F6EE37FE00E94F11E08958091EA
:10241000910124E1829FC0011124815F9F4F6EE3EF
:102420007FE00E94F11E08958091910124E1829F36
:10243000C00111248B5F9F4F6EE37FE00E94F11E6D
:1024400008958091910124E1829FC0011124805060
:1024500090406EE37FE00E94F11E0895E199FECF67
:1024600046E45FE00E94071F0895BC01809191013E
:1024700024E1829FC0011124865F9F4F0E942E128B
:102480000895BC018091910124E1829FC001112433
:10249000815F9F4F0E942E120895BC01809191018F
:1024A00024E1829FC00111248B5F9F4F0E942E1256
:1024B0000895BC018091910124E1829FC001112403
:1024C000805090400E942E1208957F928F929F928A
:1024D000AF92BF92CF92DF92EF92FF920F931F9332
:1024E000CF93DF93E199FECFE199FECF26E630E06E
:1024F0003FBB2EBBE09A8DB38F3F09F0E2C1E1995B
:10250000FECFE199FECF3FBB2EBB81E08DBB0FB666
:10251000F894E29AE19A0FBEE199FECFE199FECFDD
:1025200084E690E09FBB8EBB1DBA0FB6F894E29A8A
:10253000E19A0FBEE199FECFE199FECF85E690E0EA
:102540009FBB8EBB1DBA0FB6F894E29AE19A0FBEFC
:10255000E199FECFE199FECF3FBB2EBB81E08DBB61
:102560000FB6F894E29AE19A0FBEE199FECFE19995
:10257000FECF87E690E09FBB8EBB1DBA0FB6F894E6
:10258000E29AE19A0FBEE199FECFE199FECF88E68B
:1025900090E09FBB8EBB1DBA0FB6F894E29AE19A09
:1025A0000FBEE199FECFE199FECF89E690E09FBB97
:1025B0008EBB1DBA0FB6F894E29AE19A0FBEE1996C
:1025C000FECFE199FECF8AE690E09FBB8EBB1DBA9D
:1025D0000FB6F894E29AE19A0FBEE199FECFE19925
:1025E000FECF8BE690E09FBB8EBB1DBA0FB6F89472
:1025F000E29AE19A0FBEE199FECFE199FECF8CE617
:1026000090E09FBB8EBB1DBA0FB6F894E29AE19A98
:102610000FBEE199FECFE199FECF8DE690E09FBB22
:102620008EBB80EF8DBB0FB6F894E29AE19A0FBE95
:10263000C0E0D0E004E110E06DE7762E5AE0D52E40
:1026400045E5842E3FEA932E20E5E22E98EEF92E02
:1026500084E1A82EB4E6BB2ECC24C394C09FC00155
:10266000C19F900DD09F900D11248050904066E93D
:1026700070E00E942E12E199FECFE199FECFCE01CB
:10268000880F991F9E01F3E0220F331FFA95E1F79F
:10269000820F931F880F991F8E5F9F4F9FBB8EBB2A
:1026A0007DBA0FB6F894E29AE19A0FBEE199FECF97
:1026B000E199FECFC09FC001C19F900DD09F900DAA
:1026C00011248D5F9F4F9FBB8EBBDDBA0FB6F89470
:1026D000E29AE19A0FBEE199FECFE199FECFCE01D9
:1026E000880F991F880F991F8C0F9D1F880F991FA6
:1026F000880F991F8C5F9F4F9FBB8EBB8DBA0FB603
:10270000F894E29AE19A0FBEC09FC001C19F900D5C
:10271000D09F900D11248B5F9F4F6AE570E00E945F
:102720002E12E199FECFE199FECFC09FC001C19F5B
:10273000900DD09F900D1124895F9F4F9FBB8EBB42
:102740009DBA0FB6F894E29AE19A0FBEE199FECFD6
:10275000E199FECFC09FC001C19F900DD09F900D09
:102760001124885F9F4F9FBB8EBBDDBA0FB6F894D4
:10277000E29AE19A0FBEE199FECFE199FECFC09FA8
:10278000C001C19F900DD09F900D11249C01275F27
:102790003F4F3FBB2EBBEDBA0FB6F894E29AE19AD9
:1027A0000FBE865F9F4F6CE870E00E942E12E19989
:1027B000FECFE199FECFC09FC001C19F900DD09F79
:1027C000900D1124845F9F4F9FBB8EBBFDBA0FB647
:1027D000F894E29AE19A0FBEE199FECFE199FECF1B
:1027E000C09FC001C19F900DD09F900D1124835FA9
:1027F0009F4F9FBB8EBBADBA0FB6F894E29AE19A99
:102800000FBEE199FECFE199FECFC09FC001C19FED
:10281000900DD09F900D11249C01225F3F4F3FBB34
:102820002EBBBDBA0FB6F894E29AE19A0FBE815F53
:102830009F4F68E270E00E942E12E199FECFE1996D
:10284000FECFC09FC001C19F900DD09F900D11245D
:102850008F5E9F4F9FBB8EBBFDBA0FB6F894E29A76
:10286000E19A0FBEE199FECFE199FECFC09FC00172
:10287000C19F900DD09F900D11248E5E9F4F9FBBE6
:102880008EBBCDBA0FB6F894E29AE19A0FBEE199E9
:10289000FECFE199FECFC09FC001C19F900DD09F98
:1028A000900D11248D5E9F4F9FBB8EBBEDBA0FB66E
:1028B000F894E29AE19A0FBE2196C530D10509F04D
:1028C000CDCEE199FECF84E690E09FBB8EBBE09A2F
:1028D0008DB380939101DF91CF911F910F91FF9064
:1028E000EF90DF90CF90BF90AF909F908F907F90B0
:1028F00008959093A1018093A0018DE092E09093C0
:102900005F0280935E0210920D020895CF92DF92D3
:10291000EF92FF920F931F93DF93CF93CDB7DEB764
:1029200027970FB6F894DEBF0FBECDBF19828E0178
:102930000E5F1F4FC8016DE273E046E050E00E9459
:10294000D31EFF246E010894C11CD11CE02E012F60
:1029500016E016C0EE81FF81309731F08C819D81A9
:10296000892B11F4C6010995F394F19EB00111244D
:10297000635D7C4F8E2D902F46E050E00E94D31E69
:102980008A819B81892B31F727960FB6F894DEBF99
:102990000FBECDBFCF91DF911F910F91FF90EF90B0
:1029A000DF90CF900895EF92FF920F931F93CF93F4
:1029B000DF93EC018FE195E00E94731B2097E9F013
:1029C0008881882339F0CE010E94B51E880F880FB8
:1029D0000E94BA0F0E94B10F87FD8D5F8595859586
:1029E000E82EFF24E7FCF0940F2D1F2D8AE065E010
:1029F00041E020E20E94981B04C08FE497E00E940F
:102A0000731B84E196E00E94931BDF91CF911F918D
:102A10000F91FF90EF900895EF92FF920F931F9305
:102A2000CF93DF93EC018FE895E00E94731B209712
:102A3000A9F08881882329F0CE010E94B51E0E944A
:102A400075110E943A11E82EFF2400E010E08AE0A0
:102A500065E040E020E20E94981B04C08FE497E00C
:102A60000E94731B82E994E00E94731B8FEB94E039
:102A70000E94731B86ED94E00E94731B83E694E032
:102A80000E94931BDF91CF911F910F91FF90EF90C8
:102A90000895EF92FF920F931F93CF93DF93EC0172
:102AA00085E895E00E94731B2097A1F08881882318
:102AB00029F0CE010E94B51E0E9441120E94071209
:102AC0007C0100E010E08AE065E040E020E20E9446
:102AD000981B04C08FE497E00E94731B82E994E086
:102AE0000E94731B8EEA94E00E94731B80EE94E0B8
:102AF0000E94731B89E594E00E94931BDF91CF91A4
:102B00001F910F91FF90EF900895EF92FF920F9316
:102B10001F93CF93DF93EC018BE795E00E94731B2B
:102B20002097A9F08881882329F0CE010E94B51E44
:102B30000E9449110E941C11E82EFF2400E010E0C1
:102B40008AE065E040E020E20E94981B04C08FE428
:102B500097E00E94731B82E994E00E94731B81EA54
:102B600094E00E94731B86ED94E00E94731B83E542
:102B700094E00E94931BDF91CF911F910F91FF90E2
:102B8000EF900895EF92FF920F931F93CF93DF93EF
:102B9000EC0181E795E00E94731B2097A9F08881E2
:102BA000882329F0CE010E94B51E0E94E4110E94E4
:102BB000A911E82EFF2400E010E08AE065E040E083
:102BC00020E20E94981B04C08FE497E00E94731BD0
:102BD00089E994E00E94731B8FEB94E00E94731BC1
:102BE00086ED94E00E94731B83E694E00E94931BA1
:102BF000DF91CF911F910F91FF90EF900895EF9289
:102C0000FF920F931F93CF93DF93EC0186E695E03D
:102C10000E94731B2097A1F08881882329F0CE01A0
:102C20000E94B51E0E9435120E94FA117C0100E03C
:102C300010E08AE065E040E020E20E94981B04C0BA
:102C40008FE497E00E94731B89E994E00E94731B54
:102C50008EEA94E00E94731B80EE94E00E94731B46
:102C600089E594E00E94931BDF91CF911F910F9112
:102C7000FF90EF900895EF92FF920F931F93CF93E1
:102C8000DF93EC018BE595E00E94731B2097A9F080
:102C90008881882329F0CE010E94B51E0E94B811B8
:102CA0000E948B11E82EFF2400E010E08AE065E02E
:102CB00040E020E20E94981B04C08FE497E00E944D
:102CC000731B89E994E00E94731B81EA94E00E94DF
:102CD000731B86ED94E00E94731B83E594E00E94D1
:102CE000931BDF91CF911F910F91FF90EF9008956B
:102CF000EF92FF920F931F93CF93DF93EC0183E545
:102D000095E00E94731B2097A9F08881882329F001
:102D1000CE010E94B51E0E9406110E94CB10E82E23
:102D2000FF2400E010E08AE065E040E020E20E943D
:102D3000981B04C08FE497E00E94731B8CE894E01A
:102D40000E94731B8FEB94E00E94731B86ED94E04E
:102D50000E94731B83E694E00E94931BDF91CF9146
:102D60001F910F91FF90EF900895EF92FF920F93B4
:102D70001F93CF93DF93EC018AE495E00E94731BCD
:102D80002097A1F08881882329F0CE010E94B51EEA
:102D90000E944D120E9414127C0100E010E08AE0B3
:102DA00065E040E020E20E94981B04C08FE497E0B9
:102DB0000E94731B8CE894E00E94731B8EEA94E0DF
:102DC0000E94731B80EE94E00E94731B89E594E0DF
:102DD0000E94931BDF91CF911F910F91FF90EF9075
:102DE0000895EF92FF920F931F93CF93DF93EC011F
:102DF00081E495E00E94731B2097A9F088818823C5
:102E000029F0CE010E94B51E0E94DA100E94AD107A
:102E1000E82EFF2400E010E08AE065E040E020E2D8
:102E20000E94981B04C08FE497E00E94731B8CE8FB
:102E300094E00E94731B81EA94E00E94731B86ED6C
:102E400094E00E94731B83E594E00E94931BDF9142
:102E5000CF911F910F91FF90EF900895EF92FF9205
:102E60000F931F93CF93DF93EC018AE395E00E94C9
:102E7000731B2097A9F08881882329F0CE010E9436
:102E8000B51E0E9493100E945210E82EFF2400E00D
:102E900010E08AE065E040E020E20E94981B04C058
:102EA0008FE497E00E94731B83E894E00E94731BF9
:102EB0008FEB94E00E94731B86ED94E00E94731BDD
:102EC00083E694E00E94931BDF91CF911F910F91B5
:102ED000FF90EF900895EF92FF920F931F93CF937F
:102EE000DF93EC0182E395E00E94731B2097A1F031
:102EF0008881882329F0CE010E94B51E0E945912B4
:102F00000E9421127C0100E010E08AE065E040E0D0
:102F100020E20E94981B04C08FE497E00E94731B7C
:102F200083E894E00E94731B8EEA94E00E94731B76
:102F300080EE94E00E94731B89E594E00E94931B4D
:102F4000DF91CF911F910F91FF90EF900895EF9235
:102F5000FF920F931F93CF93DF93EC018AE295E0EA
:102F60000E94731B2097A9F08881882329F0CE0145
:102F70000E94B51E0E9465100E943210E82EFF24A8
:102F800000E010E08AE065E040E020E20E94981B4B
:102F900004C08FE497E00E94731B83E894E00E94D2
:102FA000731B81EA94E00E94731B86ED94E00E94FB
:102FB000731B83E594E00E94931BDF91CF911F91D7
:102FC0000F91FF90EF90089585E095E00E94931B8C
:102FD00081E00E94E90B08958FEF94E00E94931B1B
:102FE00082E00E94E90B08958AEF94E00E94931B0F
:102FF00080E00E94E90B0895FC01009741F090E009
:103000008081813309F491E0892F0E94A10F0895F6
:10301000CF93DF93EC0180E195E00E94731B209732
:1030200091F08881882329F0CE010E94B51E0E946C
:103030006F0F0E94660F882319F083E794E005C0A4
:1030400087E794E002C08FE497E00E94731B8DE055
:1030500097E00E94731B8AEC94E00E94931BDF911F
:10306000CF910895CF93DF93EC0180E195E00E942A
:10307000731B209791F08881882329F0CE010E944C
:10308000B51E0E94880F0E947F0F882319F083E7E6
:1030900094E005C087E794E002C08FE497E00E94C7
:1030A000731B8AEE96E00E94731B8AEC94E00E94E8
:1030B000931BDF91CF910895EF92FF920F931F938F
:1030C000CF93DF93EC0186E195E00E94731B20977C
:1030D000A9F08881882329F0CE010E94B51E0E94A4
:1030E0001E100E941510E82EFF2400E010E08AE078
:1030F00064E040E020E20E94981B04C08FE497E067
:103100000E94731B85EE95E00E94931BDF91CF9187
:103110001F910F91FF90EF900895EF92FF920F9300
:103120001F93CF93DF93EC01162F88818823A1F1A1
:10313000CE010E94B51E0E94EC0F812F0E94051047
:1031400088E995E00E94731BCE010E94B51E892B71
:1031500029F487E794E00E94931B10C00E94E30FBC
:10316000E82EFF2400E010E08AE064E040E020E286
:103170000E94981B89E594E00E94731B86E694E008
:103180000E94731B0E94FC0F882319F083E794E0D0
:1031900016C087E794E013C00E94101A64E070E044
:1031A0000E94F8217B010027F7FC0095102F8AE090
:1031B00064E041E020E20E94981B83E594E00E94D5
:1031C000931BDF91CF911F910F91FF90EF90089586
:1031D00061E00E948D18089560E00E948D180895A6
:1031E0001F9389EC93E00E94931B1092980182E94F
:1031F00091E06DE273E046E050E00E94D31E16E0DD
:103200002BC08091940190919501892B71F0C90197
:103210000E94731B8FE497E00E94731B80919401BE
:10322000909195010E94931B07C0E0919601F09147
:10323000970180E090E00995609198016F5F60933D
:103240009801619FB0011124635D7C4F82E991E098
:1032500046E050E00E94D31E2091920130919301EC
:103260002115310571F60E94CA0F8F3F21F485E5C3
:1032700097E00E94731B1F910895DF92EF92FF92D7
:103280000F931F93DF93CF93CDB7DEB764970FB63D
:10329000F894DEBF0FBECDBF10929F0189E991E087
:1032A0006DE273E046E050E00E94D31E7E01089478
:1032B000E11CF11C86E0D82E2FC0C7010E94DC1E45
:1032C000F70101900020E9F78F01015010400E191D
:1032D0001F09C7016DE072E0A8010E94E31E00977C
:1032E00059F4E0919D01F0919E01309721F1C801C0
:1032F000835F9D4F09951FC060919F016F5F609331
:103300009F016D9DB0011124635D7C4F89E991E0BF
:1033100046E050E00E94D31E6091990170919A019D
:103320006115710551F685EE93E00E94931B88EDBF
:1033300093E00E94931B64960FB6F894DEBF0FBE15
:10334000CDBFCF91DF911F910F91FF90EF90DF9054
:1033500008951F93182F0E945B1B1A30A1F01D3097
:1033600091F0E0915E02F0915F02183009F522E0E1
:10337000ED30F20769F160F13197F0935F02E0936D
:103380005E02108225C080915E0290915F028D5096
:103390009240F1F0E8F00E94861B0E943D198DE0FA
:1033A00092E090935F0280935E0210920D0210C033
:1033B00082E0ED35F80760F41083E0915E02F09151
:1033C0005F023196F0935F02E0935E0231971182C3
:1033D0001F910895DF93CF930F92CDB7DEB7E091A1
:1033E000A001F091A101CE0101960995882319F061
:1033F00089810E94A9190F90CF91DF910895A1981A
:1034000084B3816484BBA898AE9AA99808958091EA
:10341000A3018F5F8093A30108958091A201089575
:10342000CF93DF93A898AE98C0E0D0E080E0A89A50
:10343000CC0FDD1F99992196A8988F5F8D30B9F731
:10344000A89A0E94B10F8F3F39F00E94B10F9927BF
:1034500087FD9095C80FD91F999B02C0CFEFDFEF72
:10346000A898A89AA898A89AA898AE9ACE01DF9191
:10347000CF910895BC01009751F01092A30187E00D
:103480009AE10E94D4098091A3018823E1F30E946C
:10349000101A20E08F5F9F4F09F421E02093A201D2
:1034A000822F0895FC0171836083538342831782C6
:1034B0001682158214820895CF93DF93EC018C81DC
:1034C0009D81892B11F4E0E018C08E819F81E881F5
:1034D000F981E80FF91FE08101969F838E836A814D
:1034E0007B818617970720F00E94E4219F838E83BB
:1034F0008C819D8101979D838C838E2FDF91CF914D
:103500000895FC019B018481958168177907B0F4C7
:1035100086819781860F971F978386836281738147
:103520008617970720F00E94E42197838683848181
:103530009581821B930B9583848308951582148251
:103540000895FC01CB012681378162817381820F4E
:10355000931F0E94E4210190F081E02DE80FF91FF4
:1035600080810895CF93DF93EC01462F2C813D811C
:103570003093A5012093A4016A817B812617370728
:1035800010F080E011C08E819F81820F931F0E94F6
:10359000E421E881F981E80FF91F40838C819D8146
:1035A00001969D838C838FEFDF91CF9108950F93C8
:1035B0001F93CF93DF938C01EB0104C0C8010E94DD
:1035C000B21A219668816623C9F78FEFDF91CF91F8
:1035D0001F910F910895FC0140E024813581828183
:1035E00093812817390708F441E0842F0895FC01DE
:1035F00040E084819581860F971F22813381821755
:10360000930708F441E0842F0895FC018481089514
:10361000FC011582148208958091AA018093A9016A
:10362000089580E00E94701D1092A90108958536CA
:1036300028F48093A9018093AA0104C01092A901E3
:103640001092AA018091A901882311F40E94701D93
:1036500008958091A9018823A9F08091A8018F5F26
:103660008093A801853628F081E08093A8010E940C
:10367000701D9091A8018091A901891718F480E02C
:103680000E94701D08951092A8011092A901109235
:10369000AA019AE0899FB001112489E29BE10E946E
:1036A0000F0A9093A7018093A60108959093AC010F
:1036B0008093AB010895E091AB01F091AC010995C5
:1036C0000895CF93DF93EC01009739F409C0219658
:1036D000E091AB01F091AC01099588818823B9F79D
:1036E000DF91CF910895CF93DF93EC01009731F4F0
:1036F0000AC0E091AB01F091AC010995FE01219661
:1037000084918823B1F7DF91CF910895E091AB01C7
:10371000F091AC018DE00995E091AB01F091AC0125
:103720008AE0099508950E94731B0E94861B0895E4
:103730002F923F924F925F926F927F928F929F92C1
:10374000AF92BF92CF92DF92EF92FF920F931F93AF
:10375000DF93CF93CDB7DEB7A3970FB6F894DEBF54
:103760000FBECDBF6AA3242E2BA3370148014423EB
:1037700051F017FF08C0EE24FF248701E618F70870
:103780000809190902C0840173012AA1215090E09F
:10379000211091E0291B29A318A2A82EBB24CC2418
:1037A000DD24C801B701A60195010E940B22FB018F
:1037B000E750FC4F64916F8FC801B701A6019501D6
:1037C0000E940B22C901DA017C018D018EE1482E95
:1037D000512C4C0E5D1E39A023C0E114F1040105EB
:1037E0001105B9F0C801B701A60195010E940B228D
:1037F000FB01E750FC4F6491D2016C93C801B70103
:10380000A60195010E940B22C901DA017C018D01FC
:1038100003C02BA1F20120833A9408944108510877
:103820003320D9F6CE014F968C01A9A10A1B1109AC
:10383000222019F197FE05C08DE2F80182938F01D5
:103840001CC0C8010197611471048104910429F01E
:103850008C018BE2D8018C9310C08C0180E2F801BE
:1038600080830BC0E091AB01F091AC01D8018D9148
:103870008D010995BAA1B150BAA3EAA1EE2391F73F
:10388000A3960FB6F894DEBF0FBECDBFCF91DF91E8
:103890001F910F91FF90EF90DF90CF90BF90AF906E
:1038A0009F908F907F906F905F904F903F902F9060
:1038B00008959093FE018093FD0108959B01AC0152
:1038C0006050704F814F9F4FF3E0660F771F881F46
:1038D000991FFA95D1F7E4E0220F331F441F551FBB
:1038E000EA95D1F70E940B22215029B9089581E66B
:1038F00092E008958AE692E00895982F8091600200
:103900008823E1F39CB9109260020895982F80916A
:1039100060028823E1F39CB91092600281E090E09C
:1039200008951092660210926502089520E0809139
:10393000650290916602892B09F421E0822F089597
:103940001F920F920FB60F9211242F933F934F9314
:103950005F936F937F938F939F93AF93BF93EF93F7
:10396000FF936CB181E692E00E94B21AFF91EF9151
:10397000BF91AF919F918F917F916F915F914F9187
:103980003F912F910F900FBE0F901F901895682FA9
:103990008AE692E00E94B21A08951F920F920FB623
:1039A0000F9211242F933F934F935F936F937F93C5
:1039B0008F939F93AF93BF93EF93FF93809169028F
:1039C000882371F080916E0290916F02892B31F003
:1039D0008AE692E00E945C1A8CB905C010926902D6
:1039E00081E080936002FF91EF91BF91AF919F9131
:1039F0008F917F916F915F914F913F912F910F9098
:103A00000FBE0F901F90189580916E0290916F02DB
:103A1000892B99F080916902882379F481E0809361
:103A200069028AE692E00E945C1A982F80916002F7
:103A30008823E1F39CB9109260020895CF93DF933D
:103A4000EC018091630290916402892B69F080916E
:103A5000650290916602892B39F081E692E00E941E
:103A60005C1A888381E001C080E0DF91CF910895E6
:103A700081E692E06DEA71E048E250E00E94521A5D
:103A80008AE692E065ED71E048E250E00E94521A49
:103A90000895EF92FF920F931F937B018C010E9478
:103AA000381D1092FE011092FD0188ED8AB960E880
:103AB00075E280E090E00E945E1C81E080936002ED
:103AC0001092690210927302109272027894C801E7
:103AD000B7010E945E1C1F910F91FF90EF90089517
:103AE000882319F0AF9AC5980895AF98C59A08959C
:103AF00080E0089520E080910202882309F421E00B
:103B00002093020290910002992351F0222321F088
:103B100088B3892B88BB089588B39095982398BB68
:103B20000895C79A08958091FF010895282F8093E2
:103B3000FF0190910002907E90930002309101026B
:103B4000307E3093010288B38F6188BB253031F11C
:103B5000263070F42230C1F0233020F4213009F0F7
:103B600054C010C0233091F0243009F04EC010C072
:103B7000273011F12730D8F0283091F1293009F0A1
:103B800044C039C0906105C0926003C0946001C018
:103B90009860909300023093010208950E94980F5C
:103BA0009091000220910102882371F013C090933C
:103BB0000002832F826018C00E94980F909100022B
:103BC00020910102882331F09E7F90930002822F82
:103BD00081600AC09B7F90930002822F846004C0A2
:103BE00090930002832F88608093010298B38095A0
:103BF000892388BB089590930002832F806180936E
:103C0000010298B38095892388BB0895BC01C798A9
:103C100081E99DE10E94D4090895109207028091E4
:103C200000028E7F80930002809101028160809368
:103C3000010298B38095892388BB89E49EE168EEF0
:103C400073E00E940F0A9093060280930502809110
:103C500007028630E0F30895A79AAF9887B38F6B79
:103C600087BB8091000280748093000280910102E2
:103C700080748093010288B38F6B88BB8AE79DE1D3
:103C800064EF71E00E940F0A909304028093030294
:103C90000895809107028F5F809307028091070249
:103CA000833031F1843030F4813061F0823009F0BA
:103CB0005BC013C0853091F1853028F1863009F062
:103CC00053C03DC0809101028E7FC09A9091000246
:103CD0009C7F9093000282602BC0809101028D7FB7
:103CE000C19A90910002997F90930002846020C055
:103CF000809101028B7FC29A90910002937F9093F2
:103D00000002886015C080910102877FC39A90915C
:103D10000002977E9093000280610AC080910102A8
:103D20008F7EC49A909100029F7C909300028062E3
:103D30008093010298B38095892388BB0895809170
:103D400000028F7D80930002809101028F7D80931D
:103D50000102C59A88EE93E00E94061E809105023A
:103D6000909106020E944B0A0895FC01882799272A
:103D7000E89421912032E9F3293010F02E30C8F375
:103D80002B3241F02D3239F4689404C00E941C1F7C
:103D9000820F911D219120532A30C0F31EF490957B
:103DA00081959F4F0895FB01DC0102C005900D92A3
:103DB00041505040D8F70895FB01DC0105900D9269
:103DC0000020E1F70895FB01DC014150504030F044
:103DD0008D910190801919F40020B9F7881B990B77
:103DE0000895DF92EF92FF920F931F937B018C0156
:103DF000FB010995D82EC8010196F7010995982F66
:103E00008D2D1F910F91FF90EF90DF900895DF921D
:103E1000EF92FF920F931F93D72E7A018C01FA0134
:103E20000995C80101966D2DF70109951F910F9114
:103E3000FF90EF90DF9008957AE0979F902D879FF5
:103E4000802D910D11240895AEE0B0E0EAE2FFE18B
:103E50000C9456220D891E8986E08C831A8309836F
:103E60008FEF9FE79E838D839E01275E3F4FCE019C
:103E700001966F89788DA9010E94481F2F8138858E
:103E8000020F131FF80110822E96E4E00C947222A8
:103E9000ABE0B0E0EEE4FFE10C9448223C012B01E2
:103EA0005A01FC0117821682838181FD03C06FEFE6
:103EB0007FEFC6C19AE0892E1E010894211C311C97
:103EC000F3012381F20123FD859123FF81912F01CD
:103ED000882309F4B2C1853239F423FD859123FF8B
:103EE00081912F01853229F490E0B3010E943B219A
:103EF000E7CF982FFF24EE249924FFE1FF15D0F09F
:103F00009B3269F09C3228F4903259F0933291F44C
:103F10000EC09D3249F0903369F441E024C052E074
:103F2000F52A84E0F82A28C098E0F92A25C0E0E1C3
:103F3000FE2A22C0F7FC29C0892F80538A3070F4F2
:103F4000F6FE05C0989C902C1124980E15C0E89C94
:103F5000E02C1124E80EF0E2FF2A0EC09E3229F474
:103F6000F6FC6BC140E4F42A07C09C3619F450E813
:103F7000F52A02C0983649F4F20123FD959123FFFA
:103F800091912F01992309F0B8CF892F855483305F
:103F900018F08052833038F444E050E0A40EB51E8F
:103FA0005FE359830FC0933631F0933779F093353F
:103FB00009F056C020C0F5018081898342E050E0BD
:103FC000A40EB51E610101E010E012C0F501C08031
:103FD000D180F6FC03C06FEF7FEF02C0692D70E067
:103FE00042E050E0A40EB51EC6010E9430218C01B3
:103FF0005FE7F52214C0F501C080D180F6FC03C054
:104000006FEF7FEF02C0692D70E042E050E0A40E38
:10401000B51EC6010E9425218C0150E8F52AF3FE49
:1040200007C01AC080E290E0B3010E943B21EA94ED
:104030008E2D90E008171907A8F30EC0F601F7FCC3
:104040008591F7FE81916F0190E0B3010E943B21C1
:10405000E110EA94015010400115110579F7EAC00A
:10406000943611F0993669F5F7FE08C0F501208104
:1040700031814281538184E090E00AC0F501808162
:1040800091819C01442737FD4095542F82E090E0B8
:10409000A80EB91E9FE6F92257FF09C0509540951A
:1040A000309521953F4F4F4F5F4FE0E8FE2ACA0100
:1040B000B901A1012AE030E00E946721D82ED21870
:1040C00040C0953729F41F2D1F7E2AE030E01DC027
:1040D0001F2D197F9F3661F0903720F4983509F035
:1040E000ACC00FC0903739F0983709F0A6C004C0B3
:1040F00028E030E00AC0106114FD146020E130E0D7
:1041000004C014FD166020E132E017FF08C0F5017D
:10411000608171818281938144E050E008C0F501A3
:1041200080819181BC0180E090E042E050E0A40EEB
:10413000B51EA1010E946721D82ED2188FE7F82E54
:10414000F122F6FE0BC05EEFF522D91438F4F4FE2E
:1041500007C0F2FC05C08FEEF82202C01D2D01C081
:10416000192DF4FE0DC0FE01ED0DF11D808180338F
:1041700019F499EEF92208C01F5FF2FE05C003C0D2
:104180008F2D867809F01F5F0F2DF3FC14C0F0FE11
:104190000FC01E1510F09D2C0BC09D2C9E0C911A6B
:1041A0001E2D06C080E290E0B3010E943B211F5FFC
:1041B0001E15C0F304C01E1510F4E11A01C0EE2450
:1041C00004FF0FC080E390E0B3010E943B2102FF97
:1041D0001DC001FD03C088E790E00EC088E590E0B7
:1041E0000BC0802F867891F001FF02C08BE201C0E6
:1041F00080E2F7FC8DE290E0B3010E943B2106C013
:1042000080E390E0B3010E943B219A94D914C0F35B
:10421000DA94F101ED0DF11D808190E0B3010E946F
:104220003B21DD20A9F706C080E290E0B3010E94A7
:104230003B21EA94EE20C1F743CEF30166817781FA
:10424000CB012B96E2E10C946422FC0105906150B5
:1042500070400110D8F7809590958E0F9F1F08959C
:10426000FC016150704001900110D8F78095909545
:104270008E0F9F1F08950F931F93CF93DF938C0191
:10428000EB018B8181FF1BC082FF0DC02E813F811E
:104290008C819D812817390764F4E881F9810193A5
:1042A000F983E88306C0E885F985802F0995892B75
:1042B00031F48E819F8101969F838E8302C00FEF20
:1042C0001FEFC801DF91CF911F910F910895FA015F
:1042D000AA27283051F1203181F1E8946F936E7F45
:1042E0006E5F7F4F8F4F9F4FAF4FB1E03ED0B4E036
:1042F0003CD0670F781F891F9A1FA11D680F791F77
:104300008A1F911DA11D6A0F711D811D911DA11D87
:1043100020D009F468943F912AE0269F1124301997
:10432000305D3193DEF6CF010895462F4770405D32
:104330004193B3E00FD0C9F7F6CF462F4F70405DE1
:104340004A3318F0495D31FD4052419302D0A9F73C
:10435000EACFB4E0A6959795879577956795BA9536
:10436000C9F700976105710508959B01AC010A2EFC
:1043700006945795479537952795BA95C9F7620FD3
:10438000731F841F951FA01D0895629FD001739F06
:10439000F001829FE00DF11D649FE00DF11D929FE1
:1043A000F00D839FF00D749FF00D659FF00D992720
:1043B000729FB00DE11DF91F639FB00DE11DF91F44
:1043C000BD01CF0111240895AA1BBB1B51E107C0F9
:1043D000AA1FBB1FA617B70710F0A61BB70B881F95
:1043E000991F5A95A9F780959095BC01CD01089524
:1043F00097FB092E07260AD077FD04D0E5DF06D00B
:1044000000201AF4709561957F4F0895F6F7909506
:1044100081959F4F0895A1E21A2EAA1BBB1BFD0197
:104420000DC0AA1FBB1FEE1FFF1FA217B307E40793
:10443000F50720F0A21BB30BE40BF50B661F771FEB
:10444000881F991F1A9469F76095709580959095CB
:104450009B01AC01BD01CF01089597FB092E0526F4
:104460000ED057FD04D0D7DF0AD0001C38F4509589
:104470004095309521953F4F4F4F5F4F0895F6F788
:1044800090958095709561957F4F8F4F9F4F0895C0
:104490002F923F924F925F926F927F928F929F9254
:1044A000AF92BF92CF92DF92EF92FF920F931F9342
:1044B000CF93DF93CDB7DEB7CA1BDB0B0FB6F894F3
:1044C000DEBF0FBECDBF09942A88398848885F8433
:1044D0006E847D848C849B84AA84B984C884DF80A4
:1044E000EE80FD800C811B81AA81B981CE0FD11D88
:1044F0000FB6F894DEBF0FBECDBFED010895F8945E
:02450000FFCFEB
:10450200770448014F016D01740192019901B701CD
:10451200BE01DC01E3010102080226022D024B0268
:1045220052027002770295029C02BA02C102DF02B5
:10453200E60200000000008F00019700029B0003CA
:10454200B00004B60000C800257320253032640094
:00000001FF
